:100000000C9446000C9463000C9463000C94630001
:100010000C9463000C9463000C9463000C946300D4
:100020000C9463000C9463000C9463000C946300C4
:100030000C9463000C9463000C9463000C946300B4
:100040000C9463000C9463000C9463000C946300A4
:100050000C9463000C9463000C9463000C94630094
:100060000C9463000C9463000C9463000C94630084
:100070000C9463000C9463000C9463000C94630074
:100080000C9463000C9463000C94630011241FBE55
:10009000CFEFD0E1DEBFCDBF11E0A0E0B1E0E8E7F7
:1000A000F1E000E00BBF02C007900D92A030B10755
:1000B000D9F711E0A0E0B1E001C01D92A030B10776
:1000C000E1F70C9487000C940000CF93DF93CDB739
:1000D000DEB710923B0080E480933A001092380023
:1000E00010923700109235001092340010923200B6
:1000F0001092310080E28093230080E380932200FD
:100100001092620010926100DF91CF910895CBEFC1
:10011000D0E1DEBFCDBF0E946500809139009927F4
:1001200080749070009739F08FEB90913B00892399
:1001300080933B0005C080913B00806480933B002E
:100140008FE090E09A83898389819A81009729F3CF
:1001500080E593EC9C838B838B819C81009731F0AD
:100160008B819C8101979C838B83F6CF89819A81B7
:0801700001979A838983E8CF0F
:00000001FF
